:10067B00050A0000000000010F0001140102120026
:10068B000002080000021500000217000102100012
:01069B00005E
:03000B000200866A
:10008600C0E0C0F0C083C082C0D075D000C000C040
:1000960001C002C003C004C005C006C007E50B646A
:1000A6000160030202D60513E513700205127519E5
:1000B60005751ADCD39464E51264809480400E754D
:1000C60012007513000511E51170020510D3E5182D
:1000D6009405E5176480948040030201A7AE19AF2A
:1000E6001A7C007D0A1205CCC3E5119FEE6480F8E8
:1000F600E510648098501CAE19AF1A7C037DE81297
:1001060005CCAC10AD11CFCDCFCECCCE1205CC8E5A
:10011600158F16E51760030201A7E51824FE601681
:1001260014601E14602B14604924047074AD16AC60
:10013600157F010201A212069DAD16AC157F028045
:100146005B12069D7F0212069FAD16AC157F0380DB
:100156004B12069D7D647C007F027E001206A57D03
:10016600647C007F037E001206A5AD16AC157F04E5
:10017600802A12069D7D647C007F027E001206A501
:100186007D647C007F037E001206A57D647C007F73
:10019600047E001206A5AD16AC157F057E0012067C
:1001A600A5D3E5189405E5176480948050030202F0
:1001B60095AE19AF1A7C007D0A1205CCC3E5119FD6
:1001C600EE6480F8E5106480985022AE19AF1A7C70
:1001D600037DE81205CCAC10AD11CFCDCFCECCCE81
:1001E6001205CCC374649FF516E49EF515E51760F9
:1001F60003020295E51824F9601814602614603D80
:1002060014605D24046003020295AD16AC157F05EB
:100216008078E4FDFC7F05FE1206A5AD16AC157FC1
:10022600048067E4FDFC7F05FE1206A5E4FDFC7F65
:1002360004FE1206A5AD16AC157F03804DE4FDFC49
:100246007F05FE1206A5E4FDFC7F04FE1206A5E46A
:10025600FDFC7F03FE1206A5AD16AC157F02802AB3
:10026600E4FDFC7F05FE1206A5E4FDFC7F04FE12FC
:1002760006A5E4FDFC7F03FE1206A5E4FDFC7F0255
:10028600FE1206A5AD16AC157F017E001206A5AEC0
:1002960019AF1A7C007D0A1205CCD3E5119FEE64D6
:1002A60080F8E5106480984014751000751100758B
:1002B60015007516000518E51870020517D3E51820
:1002C600940AE51764809480400675170075180136
:1002D600E50C640160030203C80513E5137002050B
:1002E60012D39464E51264809480400E75120075F2
:1002F60013000511E51170020510AE19AF1A7C0046
:100306007D0A1205CCAA06AB07C3E5119BEA6480F9
:10031600F8E510648098501CAE19AF1A7C037DE88E
:100326001205CCAC10AD11CFCDCFCECCCE1205CCB4
:100336008E158F16C3E5119BEA6480F8E51064807C
:10034600984022AE19AF1A7C037DE81205CCAC109A
:10035600AD11CFCDCFCECCCE1205CCC374C89FF590
:1003660016E49EF515AD16AC157F017E001206A5A6
:10037600AD16AC157F027E001206A5AD16AC157F34
:10038600037E001206A5AD16AC157F047E0012068C
:10039600A5AD16AC157F057E001206A5AE19AF1ADF
:1003A6007C007D051205CCD3E5119FEE6480F8E54F
:1003B60010648098400C7510007511007515007555
:1003C6001600E50D640160030204950513E513703C
:1003D600020512751900751A64D39464E5126480D7
:1003E6009480400E7512007513000511E511700218
:1003F6000510AE19AF1A7C007D0A1205CCC3E511B3
:100406009FEE6480F8E51064809850367D0A7C0083
:100416007F017E001206A57D0A7C007F027E001207
:1004260006A57D0A7C007F037E001206A57D0A7C58
:10043600007F047E001206A57D0A7C007F057E00F3
:10044600802AE4FDFC7F01FE1206A5E4FDFC7F0286
:10045600FE1206A5E4FDFC7F03FE1206A5E4FDFCE4
:100466007F04FE1206A5E4FDFC7F05FE1206A5AE7E
:1004760019AF1A7C007D051205CCD3E5119FEE64F9
:1004860080F8E5106480984006751000751100D05C
:1004960007D006D005D004D003D002D001D000D0BA
:0A04A600D0D082D083D0F0D0E03235
:0A06CA0000007F067E5DDEFEDFFC0F
:0106D4002203
:0E06BB0000007F6A7E0F7D83DDFEDEFCDFFA2D
:0106C900220E
:0300830002000E6A
:10000E00C0E0C0D075D000C005C006C007E514B46E
:10001E00011720B0081206CA20B002050FD3E50F53
:10002E00648094864003750F01E514701620B0139A
:10003E001206BB20B00D751401C2B21206CAD2B29E
:0E004E00750F01D007D006D005D0D0D0E0321B
:1004B000E4F5B2F5B1F5CAF5C9758F40F589758EC9
:1004C00080758AAE758CFBD28CD2A9D2AF8012E532
:1004D0000F1460191460201460291460362404700D
:1004E00045D2B2D2B3D2CCD2CDD2B180E2E4F50AB9
:1004F000750B01F50C8008E4F50AF50B750C01F598
:100500000D800AE4F50AF50BF50C750D01F50ED218
:100510008C80BCE4F50AF50BF50CF50D750E01C2E7
:100520008C1206D580A9D2B2D2B3D2CCD2CDD2B160
:10053000E4F514F512F513F517F518758702808F99
:10005C00EE7020EF24FE6010146010146010146019
:10006C00102404700EC2B222C2B322C2CC22C2CD62
:04007C0022C2B122C9
:10065700EE7020EF24FE6010146010146010146018
:10066700102404700ED2B222D2B322D2CC22D2CD21
:0406770022D2B122B8
:08069D007F017D647C007E00FA
:1006A500C3E5139DEC6480F8E5126480985003025D
:0606B500005C1206572252
:0B06D500C2B2C2B3C2CCC2CDC2B1227F
:03000000020540B6
:0C054000787FE4F6D8FD75811A0205876B
:1005CC00C2D5EC30E709B2D5E4C39DFDE49CFCEE4A
:1005DC0030E715B2D5E4C39FFFE49EFE120602C3BA
:1005EC00E49DFDE49CFC800312060230D507C3E4B5
:0605FC009FFFE49EFE22B9
:10054C000204B0E493A3F8E493A34003F68001F211
:10055C0008DFF48029E493A3F85407240CC8C333B0
:10056C00C4540F4420C8834004F456800146F6DF7F
:10057C00E4800B010204081020408090067BE47E8E
:10058C00019360BCA3FF543F30E509541FFEE49374
:10059C00A360010ECF54C025E060A840B8E493A33B
:1005AC00FAE493A3F8E493A3C8C582C8CAC583CA66
:1005BC00F0A3C8C582C8CAC583CADFE9DEE780BE1E
:01069C00005D
:10060200BC000BBE0029EF8DF084FFADF022E4CCDC
:10061200F875F008EF2FFFEE33FEEC33FCEE9DECA5
:10062200984005FCEE9DFE0FD5F0E9E4CEFD22EDEB
:10063200F8F5F0EE8420D21CFEADF075F008EF2F35
:10064200FFED33FD4007985006D5F0F222C398FD26
:050652000FD5F0EA22C3
:00000001FF
